:100000006F10003D00000000F2010000F40100004C
:1000100000000000000000000000000000000000E0
:1000200000000000000000000000000000000000D0
:10003000CE13000000000000CE13000000000000FE
:10004000CE130000CE130000CE130000CE1300002C
:10005000C4060000CE130000CE130000CE13000033
:10006000CE130000CE130000CE130000CE1300000C
:10007000CE130000CE130000CE130000CE130000FC
:10008000CE130000CE130000CE130000CE130000EC
:10009000CE130000CE130000CE13000000000000BD
:1000A000511126C022C206C4828282441244A24058
:1000B000310182802A86014593F6150091C232955E
:1000C00085810606F5F9828000000000634E050276
:1000D00063C305042E86AA857D5515C285466378BF
:1000E000B6006356C00006068606E36CB6FE014500
:1000F00063E4C500918D558D85820582F5FA828075
:100100008682C93F2E8582823305A04063D70500D1
:10011000B305B040C1B7B305B0408682653F330533
:10012000A0408282868263C70500634905005D376F
:100130002E858282B305B040E35B05FE3305A04007
:10014000513F3305B040828200003D432A876373EC
:10015000C3029377F700BDEFADE5937606FF3D8AC6
:10016000BA960CC34CC30CC74CC74107E36BD7FE10
:1001700011E28280B306C3408A0697020000969679
:100180006780A6002307B700A306B7002306B700C1
:10019000A305B7002305B700A304B7002304B700E5
:1001A000A303B7002303B700A302B7002302B700DD
:1001B000A301B7002301B700A300B7002300B700D5
:1001C000828093F5F50F93968500D58D9396050162
:1001D000D58D61B793962700970200009696868288
:1001E000E78086FA9680C1171D8F3E96E374C3F8A8
:1001F000A5B701A0B707EFBE37E700E09387070870
:100200003CC701A07D151317050141839307F00337
:1002100063EBE700B70700209387C701AA978823FD
:100220001375F50F828001458280EFF27FE7B7E713
:1002300000E03707100023A0E7180F100000EF10B0
:10024000A04313051003EF10A04537450008130520
:1002500005FCB7040020EF10A04801449384C401BA
:10026000B38784008C2393071400A6979C233745FB
:100270000008130505FCA207DD8D2295EF10C0498B
:10028000090493070004E31DF4FCEF108040C52827
:10029000B7E700E03707100023A0E71039B5EFF209
:1002A0003FE0B7460008370400208147938606FCEC
:1002B0001304C401130600043387D7001823B305C1
:1002C000F40085071377F70F98A1E397C7FE7C30FA
:1002D0001307F00F6312F70209678147130747B44A
:1002E000930600043306F7000C223306F40085075A
:1002F0000CA2E399D7FE153F0347F403B70700208C
:1003000085461377F70F9387870163E4E60098A388
:1003100069BB23800700EDBF9307F5FF1397070123
:1003200041839307F00363EBE704EFF27FD7B7074E
:100330000020A1462A849387C7016317D5026395DD
:10034000A50289660147938646B413060004B38567
:10035000E6008821B385E700050788A1E319C7FEF9
:10036000E935EF00D04311A8BA9798236387E500D9
:100370008CA3653DA547E306F4FE05BB8280EFF242
:100380003FD223A40184239C0184A3820184238B74
:100390000184B7070040DE334145C207C18323967D
:1003A000F184EF10C02C11B3EFF29FCF1C210D4749
:1003B0007111AA8493F7F70F6374B70A1831139475
:1003C000870013740430598C9306400713F7470FC6
:1003D00005046312D702A18B99C7EF00B050AC207F
:1003E00022851D3F91A02285313DBC20631EF50270
:1003F000EF00504F15A893F7C70F130780076395B9
:10040000E7023C21228593F7F70F3EC0E53BB82079
:100410008247418B9D8B19EBB820B357F540858BF4
:100420000D83058BE386E7FC110141B13EC0EF006F
:10043000704B8247B8208544B394F400E20493776C
:100440008700E184228591C7753B458D9375F50F33
:1004500041BF4D3B93C4F4FFE98C93F5F40F49B7CA
:10046000E394E5FC13F7070F93060007E31ED7FAA2
:1004700013F777009546631AD7001C313707002021
:1004800093F7F70F2300F700A5B793F647009DE217
:10049000B706002003C506000A0575153A95420502
:1004A000418159D1A18B95C72AC0EF00B0438C3050
:1004B000024505BF9146630AD70099466309D700F4
:1004C0009D462145E312D7F6F1BF7545E1BF1D45B5
:1004D000D1BF0D3B9C3019BF8280EFF27FBCB307C8
:1004E000C5009C231307F00393F7F70F6397E70802
:1004F000130726006353B70805062A9618221C2204
:1005000085469354770013F4F707631ED400A38342
:10051000018623830186238C0186B7070020A380F0
:1005200097000D25B1A009C49307F4FF13F4F70F4A
:10053000B706002083C62600639D960283C6718697
:100540008DEA0DC81305F002753909CD054613056E
:10055000F002238CC1867D31931625003695060561
:10056000239DA186B7070020A3809700238381865F
:100570002DBE6DF8238C0186F5B713F7070C930693
:100580000004631AD70693D6574013971700918734
:10059000798B858BD98F1387E7FF1377F70F854505
:1005A00093F41600E3F5E5F6014463F7F50093874D
:1005B000D7038A0713F4F70FB707002083C7270074
:1005C0006397970283C771869DE31DC01305F002F0
:1005D000153949D905471305F002238CE1861D31F1
:1005E000131725003A950605239DA186A5BF3DF862
:1005F000238C018685BF13F7070E93060008631A44
:10060000D70213D74740058B2384E18613D73740A1
:10061000058BA387E18613D72740058B2387E186C7
:1006200013D71740058BA386E186858B2386F18639
:10063000CDBD13F7070F9306000B6315D70213D731
:100640003740058BA389E18613D72740058B238983
:10065000E18613D71740058BA388E186858B238815
:10066000F186C1B59306000A6315D70213D7374048
:10067000058BA385E18613D72740058B2385E1866B
:1006800013D71740058BA384E186858B238AF186D7
:1006900049BD13F7C70F9306C00EE31BD7EC130732
:1006A0003600E357B7EC130716002A9718230906FC
:1006B0002A96139587000C2213750530598D050570
:1006C000A1397DB57111414522C0EF007078630DED
:1006D000050C4145EF00B079B7070040DA33938746
:1006E000C18482234207418333048740420441800E
:1006F000CD4663FB860A37150140C1451305054009
:100700009AA3EF10600C4DE10967130707719387F7
:1007100081846377870023A00700239C018469A05C
:10072000984385466305D70A25C38946E315D7FE56
:10073000138661841822133414050607598C137428
:10074000F40F9386418400A2982205071377F70FD0
:1007500098A2A146631AD70493865184982295459E
:1007600063E1E50298229375F70F1387150013775D
:10077000F70F98A214221387018593F6F60F2E9790
:1007800014A3054798C30DA0930600051387818520
:1007900063E086021E239306900F63E7F6001E2394
:1007A0008507C207C1831EA30244110173002030D4
:1007B00016232546637AD600894694C32382018492
:1007C00023830184A382018423100700F1BF9306D1
:1007D000000563F98600094798C3238201842383B7
:1007E0000184D9B7238BE18423A00700239CE184F3
:1007F00065BFEFF2FF8A130141FC0545EF102000B1
:10080000EF003036693CEF00700285451305500259
:10081000EF10C00789653146138485B208109385AF
:1008200085B2EF102023371501400C101305054049
:10083000EF00D07191450D45EF00507A4146930588
:10084000C4006810EF1000216810EF00D059930722
:1008500040117C86680085473EC823070100EF00F1
:10086000707A85450545EF104004B707002003A5C1
:100870004701B7450F0093850524EFF0BF857D152F
:10088000C167FD17E8824C08370500403ECC231BAA
:100890000100230E0100EF102003854537050040BD
:1008A000EF104017B7070040C23342044180B7073A
:1008B0000040DE331307703E818FC207C183637827
:1008C000F7001304843E42044180EF00F00883C720
:1008D000618593F7F70FE1DFB7E700E03707100016
:1008E00023A0E7180F10000083C55184814793F4BB
:1008F000F50F9386018513F6F70F63669604238B35
:100900000184A3820184B7E700E03707100023A029
:10091000E710814681471387F4FF63CEE7027C1816
:100920003E97834787FCE394D7F88947E3F197F82C
:100930001C821307000793F6070F6397E602A6854C
:1009400048009D34ADB73386D700082250003E964C
:1009500008A285074DB770183E96034686FC8507AA
:1009600093F7F70FB18E55BF93F7070C13070008E5
:100970006395E70048008D361DBF7545EFF09F88F1
:100980001375050215C58D47E383F4F21C824545B6
:100990003EC0EFF03F878247E39BA7F09C8249452A
:1009A0003EC0EFF03F868247E393A7F0094611A8C7
:1009B0001C8205453EC0EFF0FF8482470546E39860
:1009C000A7EEA6854800113EDDB5EFF26FED1301ED
:1009D000C1FD854513054020EF00506B3165EF00E8
:1009E000B0693715014099478A85130505807C80D9
:1009F000231101002312010023130100231401001D
:100A000023150100EF009054614681456800EFF026
:100A1000CFF337240140B7070E003ECC6C0085476A
:100A2000130504402300F102EF00902585451305CE
:100A30000440EF00D02913050440EF00502A93042E
:100A400004402685EF00502A6DFD1305044037242D
:100A50000140EF00F029130404402285EF00F02943
:100A60006DFD130141026FF04FE4EFF26FE33724A5
:100A70000140AA859146054613050440EF00F02980
:100A8000854513050440EF00D027930404408945B1
:100A90002685EF00B03465DD13050440EF00903388
:100AA0006FF0AFE0EFF2CFDFB7370140138407C03C
:100AB00083A747C351112AC43EC05C5C4E342285D3
:100AC0003EC28505C205C181EF0050784E342285B3
:100AD0008505C205C181EF00B07713055003EFF023
:100AE0006FF2B7070040DA33931725003E954207AF
:100AF00041830605B7060040DE32998FC207C183E5
:100B0000E3CCA7FE11448144A247054591E301458A
:100B1000A93F1307F4FF1374F70FAA9475F42C8000
:100B200037340140130504C0EF0050722C821305C6
:100B300004C0EF00F07113D524004205418131015A
:100B40006FF0AFD6EFF2CFD5B70700204111754552
:100B500083C42700EFF00FEB058919C193C414007B
:100B600003C48186938781863EC211C81305100293
:100B700099E013052002EFF0EFE81374F50F83C737
:100B8000C18681CB13053002EFF0CFE7498C137497
:100B9000F40F83C7D18681CB13054002EFF08FE6B7
:100BA000498C1374F40F83C7E18681CB130550027F
:100BB000EFF04FE5498C1374F40F83C7F18681CBB6
:100BC00013056002EFF00FE4498C1374F40F83C730
:100BD000018781CB13057002EFF0CFE2498C1374CB
:100BE000F40F83C7118781CB13058002EFF08FE1EB
:100BF000498C1374F40F83C7218781CB13059002AE
:100C0000EFF04FE0498C1374F40F83C7318781CB29
:100C10001305A002EFF00FDF498C1374F40F83C7A4
:100C2000418781CB1305B002EFF0CFDD498C1374FF
:100C3000F40F83C7918681CB1305C002EFF08FDCE0
:100C4000498C1374F40F83C7A18681CB1305D0029E
:100C5000EFF04FDB498C1374F40F83C7B18681CB5F
:100C60001305E002EFF00FDA498C1374F40F1376DA
:100C70001400894537150140EF00B0351356144074
:100C8000058A914537150140EF00B03413562440D2
:100C9000058AC14537150140EF00B0331356344083
:100CA000058A9305000237150140EF009032135674
:100CB0004440058A9305000837150140EF00703164
:100CC00013565440058A9305000437150140EF0080
:100CD0005030B7370140938707C0DE377945C207E8
:100CE000C1833EC0EFF00FD28947631DF5029247E2
:100CF0009C2395C7824781451384170099C0A2851C
:100D00000144C205B7340140C181138504C0EF001E
:100D1000F05393150401C181138504C001A201445D
:100D20008145C5B70945EFF0EFCD03C771869387BD
:100D300071863EC42A84014555CB83C7818702C290
:100D400089CB13050003EFF0EFCB93170501C183A7
:100D50003EC21545EFF00FCB13170501418319452E
:100D60003AC6EFF02FCA3247931705018546C18373
:100D700063E4E6001307F00F854663EBF600B30665
:100D8000874093D7F601B6978587A297C207C1839C
:100D9000A2468C2285466398D5089247A2971305F0
:100DA00020033EC2EFF00FC692471DC12247142315
:100DB0000547637FD70003A5C185AA9763C987004C
:100DC0003E849307F00F63D487001304F00FA287CB
:100DD0003E859307F00F63F4A7001305F00F8245DB
:100DE000EFF04FAD9305F00FEFF0CFAE8247024723
:100DF0003385A74013041700931705014204C183EC
:100E00004180BDC0A28537340140130504C03EC0F7
:100E1000EF00D0438247130504C0BE85EF00504366
:100E200041016FF08FA89306F00363EFB60033859E
:100E30008740FD15EFF00FA89305E003EFF00FA931
:100E400092472295AA97A1BF3305F740938515FCD9
:100E50003EC6EFF02FA69305F003EFF02FA7B247A1
:100E60001247AA97BA9725BFB7340140BE851385AC
:100E700004C0EF00B03DA28545B5EFF26FA241116D
:100E80002945EFF02FB803C67186938771863EC25D
:100E90001307E6FF2AC01377F70F9306B007938472
:100EA000C18563E5E60009CD636CA600984011C7D3
:100EB00023A0018623A00400713141016FF0EF9E51
:100EC0009386C1878C22138701866385C500232002
:100ED000070090A2B7060020754503C42600EFF076
:100EE0006FB2058919C1134414002285653E9247EB
:100EF0002A849305F00794231395A600158DEFF02F
:100F0000EF9C3304854013053003EFF0AFAF2AC6E2
:100F100013054003EFF00FAFB246A2852AC4368511
:100F2000EFF04F9993054006EFF04F9A1387018633
:100F30001043AA862243329409661306067163544D
:100F4000860010C339A079761306068FE34BC4FEE2
:100F500000C30C431A8536C4EFF0CF959305803E4D
:100F6000EFF0CF96A2468247B305D5008CC081CF63
:100F70009247882382473385A740EFF0AF9382459D
:100F8000EFF0CF9488C09440130780076354D700D4
:100F900098C01DB7130780F8E3CCE6FE31BFEFF22F
:100FA0002F902545EFF00FA6937775000547638BCB
:100FB000E70609471304007D638AE7000D47130421
:100FC000401F6385E7002164130404D0218911C107
:100FD0000580B707002083A44701A2852685EFF08E
:100FE0006F8FC167938787DE814563F4A7008D808B
:100FF0009D45B73701400546138507C0EF007024B3
:10100000A2852685EFF00F8D9305F5FFB7370140D8
:10101000C205C181138507C0EF001023EFF09FB216
:101020006FF0AF880964130404F44DB7EFF24F87F3
:10103000130181FD854513055003EF00300505655B
:10104000854513050580EF007004EFF01F98C14738
:101050003ECA85473EC86C009307600F37150140B4
:101060007C8623170100DD25371501409147614437
:101070006C00130505407C8622CAC92DA1476C006F
:10108000371501407C8622CAD125373401409307A9
:10109000B05D8A85130504C03EC202C0230401006E
:1010A000EF009002C167938707062C08130504C060
:1010B0003ECC02CE02D002D2EF00F0052C08130580
:1010C00004C0EF00F00B130504C08545EF001016B7
:1010D0008545130504C0EF00F013D13513018102DB
:1010E0006FE0BFFCEFE2DFFBB7070040D6330567D8
:1010F000B7040040C206C18213077738DE30958FEF
:10110000C207C183E37CF7FE05469305600F3715E0
:101110000140C125373401408355C4C2130404C0C3
:1011200022858505C205C181EF00501281452285C7
:10113000EF001012D630096737060040C206C182A0
:101140001307F7705E32958FC207C183E37CF7FE09
:10115000EFF05F9F6FE07FF5EFE29FF49387618789
:101160009A23611119C37D179AA3138781871C23C2
:1011700091CF9386A1879E2291CBFD17C207C18391
:101180009EA289E723000700EFF0DF9B37060020CF
:10119000B70700201306260083C517001C221384FE
:1011A0007186638CB70A182049C78547014710200C
:1011B0006304E6049385E18796213EC23AC0850622
:1011C00096A19384E1876370E60A0D45EFF08F8363
:1011D0000247924799C311E109459E200A0563CD54
:1011E000A7001C2063F7E708850793F7F70F1CA0FB
:1011F00023900400EFF01F9513052003EFF08F807C
:1012000015C51820854763F3E70213056003EFE077
:101210007FFF11E10545138741861E234205418169
:101220008507C207C18363F8A7041EA321016FE0ED
:10123000DFE7938601889E221305900F8507C2077A
:10124000C1839EA2E373F5F63AC00CA22390060078
:10125000EFF05F8F8547024799BF03C761862390F0
:1012600001888147A9B71145EFE0DFF992470247AE
:1012700095B7FD179DBF23100700EFF01FC07DB786
:10128000EFE21FE2371402401C403707FFF84145E8
:1012900093E717001CC05C40F98F5CC01C40370707
:1012A000F7FE7D17F98F1CC01C403707FCFF7D1728
:1012B000F98F1CC05C4041777D17F98F5CC0B70780
:1012C0009F001CC44D231C4C93E707021CCCB7178E
:1012D000014003A70740938607401377F7F023A048
:1012E000E74003A707401367070823A0E7408947A3
:1012F0009CCAB7F7FF1F03C5477D9307F00F630430
:10130000F5007D898D23B72702409843C176FD16ED
:10131000719B98C398431367170098C3B71702408F
:10132000D843D8C3D843758FD8C3D843B706000174
:10133000D8C39843558F98C3984393166700E3DD4D
:1013400006FED843B7160240719BD8C3D843136733
:101350002700D8C32147DC42B18BE39EE7FE6FE054
:10136000DFD4EFE2FFD3371702405C43370400209D
:101370009146B18B130444016385D700A146638273
:10138000D704B7376E01938707601CC0B7160240B9
:10139000DC420840918313F7F700B70700209387DA
:1013A0004700BA978C23DC4293F5F50F93F70708B3
:1013B0003357B50081E7EFE0FFD12A8718C06FE00F
:1013C000DFCE5C43B777DC02938707C07DBF01A007
:1013D00097F1FF1F93818144138181FE1305000A59
:1013E00097F5FF1F938505C217F6FF1F130686C1E9
:1013F00063FAC5008322050023A05500110591055D
:10140000E3EAC5FE170500001305057897F5FF1FF1
:10141000938545BF17F6FF1F130646C063FAC50044
:101420008322050023A0550011059105E3EAC5FEBE
:1014300017F5FF1F130585BE938581886377B50077
:10144000232005001105E36DB5FEB722000093824D
:101450000288739002308D427390428097F2FFFFB2
:10146000938242BA93E2320073905230EFF05FE120
:1014700097F2FFFF9382223873901234730020306A
:101480005C413707F1FF1307F7EF7D8FDC41944193
:10149000A207D58FD98F5CC11C4537F7F1FF130721
:1014A000D77FD4457D8F9C49D58F94458606D58FAF
:1014B000D98F1CC55C55370710FF7D177D8FDC2940
:1014C000FD1793F7F70FD207D98F5CD582801C45A3
:1014D00089C593E717001CC58280F99BEDBF1C45A9
:1014E00093E787001CC5828008450D8105898280AD
:1014F0001C4593E747001CC5828008450981058982
:1015000082801C4591C537075000D98F1CC5828049
:101510003707B0FF7D17F98FD5BFA54763F8B7042C
:10152000138765FF931717008322C500BA971D43E1
:101530003313F3001343F3FF33735300B397F600F1
:10154000B3E767005CC5994763E3C7047D1693174B
:1015500026003E965859FD47B397C70093C7F7FF3B
:10156000F98FB395C500DD8D4CD982809397150016
:1015700003230501AE971D473317F7001347F7FF05
:1015800033776700B397F6005D8F18C96DBFB14719
:1015900063E2C7026516931726003E961859FD4769
:1015A000B397C70093C7F7FFF98FB395C500DD8DDB
:1015B0000CD982804D161317260054553A96FD47D4
:1015C000B397C70093C7F7FFF58FB395C500DD8DBF
:1015D0004CD58280684542054181828008416D8DED
:1015E0003335A00082805841032305004C4537065F
:1015F0000140930706403E979346F3FFB1C583250C
:101600000640F58D2320B640D043F18ED4C3144359
:10161000B3E6660014C3184190479346F7FF758EF2
:1016200090C7D047F18ED4C7144541466399C60090
:101630009447D98E94C7D447558FD8C78280B69720
:101640009443558F98C382801C43F58F1CC38280BE
:10165000B70701401387074083A70740584B698F9E
:1016600009C77D8D3335A000828001458280B70790
:10167000014023AAA7408280B70767453727024069
:10168000938737125CC3B797EFCD9387B79A5CC344
:101690008280372702401C4B93E707081CCB8280CF
:1016A000B7270240C8C78280372702405C470545FC
:1016B000858B91E748474189133515000D058280D8
:1016C000EFE21F9E2A84CD3785476318F50019E0A5
:1016D000154529A0D13F7D14C5BF7DD86FE0FF9C83
:1016E000EFE21F9CAA8437050B00D93F9147631393
:1016F000F502372402401C4837050B0093E727000A
:101700001CC844C81C4893E707041CC8553F1C4824
:10171000F59B1CC86FE07F99EFE29F987111AA8436
:1017200009652EC0713F91478245631EF50037243D
:1017300002401C48096593E717001CC88EA0493772
:101740001C48F99B1CC811016FE03F96944593F724
:10175000060193F2F60081C7DC41B3E2F20083D3C5
:10176000050093F7F30FA5C303230500611122C2FF
:1017700026C0814713048002930480040547331672
:10178000F70033F7C3006312E602939527003D4745
:101790003317B7001347F7FF33736700B395B200F1
:1017A00033E36500639D860050C985072147E397B1
:1017B000E7FC124423206500824421018280E396E5
:1017C00096FE10C9DDB7828008456D8D3335A000C7
:1017D000828019C20CC982804CC9828037070140BF
:1017E000144786058D47B397B70093C7F7FFF58F6A
:1017F0001CC71C47B315B500DD8D0CC7828023A222
:10180000A188828083A64188854718216390F602CB
:101810001C31639CD7023C219A0793E707F8B7E68F
:1018200000E093F7F70FBA962380F640854693576A
:1018300057003397E600544189CE938707048A07FF
:10184000B7E600E0B69798C38280EDF33C219A0793
:10185000F9B793870706B7E600E08A07B69798C3FB
:101860000F1000008280371702401C430E0593F7CB
:1018700077F05D8D08C38280B7160240DC42417765
:101880001307F77FF98F5D8DC8C2828099C537171E
:1018900002401C4F5D8D08CF8280B7170240984FE1
:1018A0001345F5FF798D88CF828099C5371702409F
:1018B0005C4F5D8D48CF8280B7170240D84F1345EB
:1018C000F5FF798DC8CF82801E213737014013077D
:1018D00007C0C207C1836306E500370700406316EF
:1018E000E500BA2193F7F7F8D98FFA2193F7F7CFEC
:1018F000C207C183D98F1EA1DE215EB59E211EB510
:10190000B7370140938707C06314F5009C251EB9C3
:1019100085475EA982801E31922103D32500C2072C
:10192000C183F99BC207C1831EB11E3156211A2DF6
:10193000C207C183420741831377C7F8518F9225AD
:10194000F59BC20633666600D18F37360140130619
:1019500006C0C1826310C502B225DD9B03D3E5003A
:10196000D18FD221ED9B93F6F6CFD18FD22533665E
:101970006600D18E56A11AADFA2158D91EB18280C7
:101980001E31922103D38500C207C18393F7F7EF7D
:10199000C207C1831EB11E3156215A2DC207C18311
:1019A000420741831377C7F8518FB22193F7F7DFCE
:1019B000C206336666002206D18F13960701B73739
:1019C0000140938707C0C1824182631FF502FD7702
:1019D0009387F77FF18FB22503D3C5002206D18FFD
:1019E000D221C207C183220693F7F7BFD18F139686
:1019F0000701F577FD17FD8EFE254182B3E76700ED
:101A00009207DD8EC206C182FE2156A15AAD5CDD71
:101A100012B182801E2189C593E717001EA1828022
:101A2000C207C183F99BC207C183CDBF8357450459
:101A300091C52167D98F2312F5048280C607C5831B
:101A4000DDBF0EB552A982804EB582804CD982800E
:101A50004CDD8280B3C7A5008D8B3307C50081E7BD
:101A60008D4763E7C702AA87637EE50A942185074D
:101A70008505A38FD7FEE3EBE7FE828094218507DF
:101A80008505A38FD7FEE3EBE7FE024411018280B8
:101A900093763500AA8789CA942185078505A38F87
:101AA000D7FE93F63700C5BF9376C7FF138606FEB1
:101AB00063F5C706711122C0C04903A3050083A3C3
:101AC0008500C0CB804D23A0670003A3450080CFD5
:101AD000C04D23A2670083A2C50003A3050193851F
:101AE0004502C0CF03A4C5FF23A4770023A6570057
:101AF00023A867009387470223AE87FEE3EEC7FA69
:101B0000E3F3D7F890419107910523AEC7FECDBF0F
:101B100090419107910523AEC7FEE3EBD7FEE3E7C3
:101B2000E7F48280828000001000000001000000C5
:101B30000400000010000000000000001000000081
:101B40000100000003000000FF000A9C00400000AC
:101B500000000000C0800000000000000000000045
:101B60000200000001020408102000000000000034
:101B70000000000000000A030E1400000000000036
:041B80000000000061
:101B84000101010001020304050607080102030420
:081B940005060708006CDC02E5
:00000001FF
